:100000000C945A000C9477000C9477000C947700B1
:100010000C9477000C9477000C9477000C94770084
:100020000C9477000C9477000C9477000C94770074
:100030000C9477000C94AB070C9477000C94770029
:100040000C9472080C9477000C9477000C94770051
:100050000C9477000C9477000C9477000C94770044
:100060000C9477000C947700000024272A000025C8
:10007000282B000023262904040404040404040299
:100080000202020202030303030303010204081035
:100090002040800102040810200102040810200002
:1000A0000000070002010000030406000000000039
:1000B0000000000011241FBECFEFD4E0DEBFCDBF93
:1000C00011E0A0E0B1E0ECEBFBE102C005900D9285
:1000D000A430B107D9F711E0A4E0B1E001C01D924E
:1000E000AE3CB107E1F70E9408070C94DD0D0C94BB
:1000F00000008EBD0DB407FEFDCF8EB59927089583
:10010000E82FFF2783E0EE0FFF1F8A95E1F7EC5FF2
:10011000FE4FE60FF11D40830895E82FFF2793E07F
:10012000EE0FFF1F9A95E1F7EC5BFE4FE60FF11D16
:1001300040830895E82FFF2723E0EE0FFF1F2A9545
:10014000E1F7EC57FE4FE60FF11D408308950F9342
:10015000A82FBB27772733E0AA0FBB1F3A95E1F7FB
:10016000FD01EC5FFE4FE60FF71F4083FD01EC5BE6
:10017000FE4FE60FF71F2083AC57BE4FA60FB71FE9
:100180000C930F910895CF93DF93582F20E030E028
:100190000BC059936D9341938F5F8830D1F72F5FD8
:1001A0003F4F2830310589F0C90173E0880F991F4E
:1001B0007A95E1F7EC01CC5FDE4FDC01AC5BBE4F22
:1001C000FC01EC57FE4F80E0E4CFDF91CF91089522
:1001D0004F925F926F927F928F929F92AF92BF9257
:1001E000CF92DF92EF92FF920F931F93D82EC62EDD
:1001F000CA0168E671E00E94420D7C016CE370E088
:100200000E94420D882777FD8095982F0E94080C48
:100210004B015C010027F7FC0095102FC801B701C6
:100220000E94080C20E030E040E752E40E946D0B91
:10023000A50194010E94080B9B01AC0160E070E0F5
:1002400080E89FE30E94080B7B018C019B01AC01BD
:1002500060E070E080E89FE30E94080B2B013C0106
:1002600020E030E040E050E0C501B4010E94430CC2
:10027000882339F45301420160E070E080E89FE395
:1002800016C020E030E040E85FE3C501B4010E9401
:10029000430C8823B9F4C801B7010F2EF0E08F2E6C
:1002A000F0E09F2EF0E8AF2EFFE3BF2EF02D0F2ED3
:1002B000F0E04F2EF0E05F2EF0E06F2EF0E07F2EAA
:1002C000F02D5BC020E030E040E050E4C501B40117
:1002D0000E94430C882379F460E070E080E090E0B5
:1002E0000F2EF0E08F2EF0E09F2EF0E8AF2EFFE310
:1002F000BF2EF02D42C020E030E040E450E4C501C4
:10030000B4010E94430C882339F44701580160E08E
:1003100070E080E090E016C020E030E040E850E47B
:10032000C501B4010E94430C8823B9F4C301B20192
:100330000F2EF0E08F2EF0E09F2EF0E0AF2EF0E0D9
:10034000BF2EF02D0F2EF0E04F2EF0E05F2EF0E8E4
:100350006F2EFFE37F2EF02D10C02701380160E0E3
:1003600070E080E89FE30F2EF0E08F2EF0E09F2EEC
:10037000F0E0AF2EF0E0BF2EF02D0D2D1127DD2483
:10038000A3E0000F111FAA95E1F7F4E0EF2EF1E0D2
:10039000FF2EE00EF11EEC0CFD1C20E030E048EFDB
:1003A00051E40E94C00C0E94DA0BF7016083E4E480
:1003B000EE2EE1E0FE2EE00EF11EEC0CFD1C20E026
:1003C00030E048EF51E4C501B4010E94C00C0E9426
:1003D000DA0BF70160830C571E4F0C0D1D1D20E03A
:1003E00030E048EF51E4C301B2010E94C00C0E940A
:1003F000DA0BF80160831F910F91FF90EF90DF906F
:10040000CF90BF90AF909F908F907F906F905F90B4
:100410004F900895DF92EF92FF920F931F93CF9327
:10042000DF937C0100E010E00EC0A7016C2F8D2D42
:100430000E94E8002196C830D105B9F70F5F1F4F21
:100440000830110521F0D02EC0E0D0E0EECFDF91D2
:10045000CF911F910F91FF90EF90DF900895FF9241
:100460000F931F93CF93DF93F82E8B01C0E0D0E062
:10047000A8016F2D8C2F0E94E8002196C830D1056D
:10048000B9F7DF91CF911F910F91FF900895FF92DF
:100490000F931F93CF93DF93F82E8B01C0E0D0E032
:1004A000A8016C2F8F2D0E94E8002196C830D1053D
:1004B000B9F7DF91CF911F910F91FF9008950F939E
:1004C0001F93CF93DF93C0E0D0E000E010E0B801CD
:1004D0008C2F0E942F0221960E5C1F4FC830D10531
:1004E000B1F7DF91CF911F910F910895CF92DF92D5
:1004F000EF92FF920F931F93CF93DF936C010091C4
:10050000C4011091C501E801EE24FF24BE018E2D27
:100510000E942F020894E11CF11CCC0DDD1D88E027
:10052000E816F10499F70F5F1F4F1093C501009370
:10053000C401DF91CF911F910F91FF90EF90DF9059
:10054000CF9008958F929F92AF92BF92CF92DF92F9
:10055000EF92FF920F931F93CF93DF93982E862EE7
:100560005A01992713E0880F991F1A95E1F7B4E013
:10057000EB2EB1E0FB2EE80EF91E8C010C5B1E4F3A
:10058000EC01CC57DE4FCC24DD24882D99270C2C90
:1005900002C0959587950A94E2F780FF06C0A501F1
:1005A0006C2D892D0E94E80005C0F7011082F8012A
:1005B000108218820894C11CD11C0894E11CF11C03
:1005C0000F5F1F4F2196F8E0CF16D104F1F6DF91AF
:1005D000CF911F910F91FF90EF90DF90CF90BF9040
:1005E000AF909F908F9008950F931F938C01AC0153
:1005F00060E080E00E94A202A80160E081E00E9429
:10060000A202A80166E682E00E94A202A80160E0C0
:1006100083E00E94A202A80168E184E00E94A20295
:10062000A80169E985E00E94A202A80162E486E0CF
:100630000E94A202A8016CE387E00E94A2021F911F
:100640000F9108950F931F938C01AC0160E080E03F
:100650000E94A202A80166E681E00E94A202A8010F
:1006600066E682E00E94A202A80160E083E00E94A8
:10067000A202A80168E184E00E94A202A80169E93F
:1006800085E00E94A202A80162E486E00E94A20224
:10069000A8016CE387E00E94A2021F910F910895C8
:1006A0000F931F938C01AC0166E381E00E94A202CC
:1006B000A8016FE782E00E94A202A8016FE783E031
:1006C0000E94A202A8016EE384E00E94A202A80197
:1006D0006CE185E00E94A202A80168E086E00E9429
:1006E000A2021F910F9108958CB580658CBD8CB5C9
:1006F0008C7F8CBD8DB58EB58DB581608DBD089517
:10070000E1EBF0E0808187608083A0EBB0E08C912A
:100710008C7F8C938081877F8083E0E7F0E080810D
:10072000816080831092B20078940895E1E8F0E04F
:1007300080818D7F80838081856080838081877EBA
:100740008083E0E8F0E080818C7F8083EFE6F0E05A
:100750008081816080838FEC9EEF909385008093F1
:10076000840078940895CF92DF92EF92FF920F93D6
:100770001F938C01C62EAC0160E080E00E94A202B3
:10078000A80160E081E00E94A202A80160E082E08E
:100790000E94A202A80168E183E00E94A202A801CF
:1007A00068E184E00E94A202A80160E085E00E9466
:1007B000A202A80160E086E00E94A202A80160E017
:1007C00087E00E94A202DD24EE24FF24C701B601C7
:1007D0000E942209A80160E080E00E94A202A80114
:1007E00060E081E00E94A202A8016CE382E00E9426
:1007F000A202A80164E283E00E94A202A80164E2CE
:1008000084E00E94A202A8016CE385E00E94A2029B
:10081000A80160E086E00E94A202A80160E087E0F3
:100820000E94A202C701B6010E942209A80160E04D
:1008300080E00E94A202A8016EE781E00E94A2026D
:10084000A80162E482E00E94A202A80162E483E0BF
:100850000E94A202A80162E484E00E94A202A80110
:1008600062E485E00E94A202A8016EE786E00E9491
:10087000A202A80160E087E00E94A202C701B601BF
:100880000E942209A8016FEF80E00E94A202A80145
:1008900061E881E00E94A202A80161E882E00E9472
:1008A000A202A80161E883E00E94A202A80161E817
:1008B00084E00E94A202A80161E885E00E94A202F1
:1008C000A80161E886E00E94A202A8016FEF87E01C
:1008D0000E94A202C701B6010E94220940E060E026
:1008E00080E00E94C3001F910F91FF90EF90DF9076
:1008F000CF900895AF92BF92CF92DF92EF92FF9286
:100900000F931F93CF93DF93EC01C62E5A01DD2482
:100910001BC075010027F7FC0095102FC801B70117
:100920000E942209CE010E942203C801B7010E9441
:100930002209CE010E94F402C801B7010E942209D7
:10094000CE010E942203D394DC1419F7DF91CF91DA
:100950001F910F91FF90EF90DF90CF90BF90AF90DD
:100960000895CF93DF93C0E0D0E0AE0166E381E06D
:100970000E94A202AE016FE782E00E94A202AE01D5
:100980006FE783E00E94A202AE016EE384E00E9462
:10099000A202AE016CE185E00E94A202AE0168E015
:1009A00086E00E94A2026CE070E080E090E00E948D
:1009B0002209609681E0C037D807B9F6DF91CF9160
:1009C0000895DF92EF92FF920F931F93CF93DF93DF
:1009D000EE24FF2422C0A7016C2F8D2D0E94E80079
:1009E00065E070E080E090E00E9422092196C83026
:1009F000D10589F70F5F1F4F0830110551F480E2D0
:100A000090E0E80EF91E90E8E91691E0F90641F051
:100A100004C0D02EC0E0D0E0DECF00E010E0F9CF7F
:100A2000DF91CF911F910F91FF90EF90DF9008958C
:100A3000EF92FF920F931F93CF93DF93C0E0D0E02C
:100A4000EE24FF248701C801B7010E94080C0E9410
:100A5000D50BDC01CB010E940A0264E070E080E06B
:100A600090E00E942209239683E090E0A0E0B0E0AD
:100A7000E80EF91E0A1F1B1F91E0C836D90719F7A7
:100A8000DF91CF911F910F91FF90EF9008950F93F9
:100A90001F93CF93DF9300E010E03DC049934D9347
:100AA00041938F5F8830D1F72F5F3F4F283031055A
:100AB00009F564E070E080E090E00E9422090F5F99
:100AC0001F4F00321105E1F126C019931D931193B8
:100AD0008F5F8830D1F72F5F3F4F28303105F9F411
:100AE00064E070E080E090E00E94220911501F3F16
:100AF00059F127C0C90153E0880F991F5A95E1F7B2
:100B0000EC01CC5FDE4FDC01AC5BBE4FFC01EC576F
:100B1000FE4F80E0C3CF402F20E030E0EBCFC90193
:100B200003E0880F991F0A95E1F7EC01CC5FDE4FD7
:100B3000DC01AC5BBE4FFC01EC57FE4F80E0C5CF43
:100B40001FE120E030E0EBCFDF91CF911F910F91BB
:100B50000895AF92BF92CF92DF92EF92FF920F93E0
:100B60001F9368E671E080E090E00E94490A5B0113
:100B70006C0168E070E080E090E00E94490A7B012F
:100B80008C0168E070E080E090E00E94490ADC019E
:100B9000CB01A5016E2D0E94E8001F910F91FF90DF
:100BA000EF90DF90CF90BF90AF900895CF93DF93F9
:100BB000C0E0D0E00E9447052196C430D105D1F7AE
:100BC000C0E0D0E00E9418052196C230D105D1F7CF
:100BD000C0E0D0E08EE190E00E947602219683E0B2
:100BE000C83ED807B9F7C0E0D0E00E945F02219666
:100BF000C436D105D1F7C0E0D0E080E590E00E9496
:100C00000A022196CA30D105C1F70E94E10440E0F2
:100C100060E080E00E94C300C0E0D0E080E090E0AF
:100C20000E9450032196CA3FD105C1F7C0E0D0E031
:100C30000E94B1042196C430D105D1F7C0E0D0E0C4
:100C40000E94A905219687E2C031D807C9F744E67A
:100C500050E068E088EC90E00E947A0464EC79E06F
:100C600080E090E00E94220966E98CE291E00E9417
:100C7000B303DF91CF910895AF92BF92CF92DF92ED
:100C8000EF92FF920F931F93CF93DF93AA24BB247D
:100C90007CC08881C81650F481E090E0022E02C02A
:100CA000880F991F0A94E2F78095D8228081C81690
:100CB00050F481E090E0022E02C0880F991F0A9440
:100CC000E2F78095E8228C91C81650F481E090E01C
:100CD000022E02C0880F991F0A94E2F78095F8222D
:100CE0002F5F3F4F2196119631962830310589F6B6
:100CF00060E08AE00E94BD09FEBC0DB407FEFDCF96
:100D00008EB5EEBC0DB407FEFDCF8EB5DEBC0DB4C6
:100D100007FEFDCF8EB581E090E0002E02C0880F67
:100D2000991F0A94E2F78EBD0DB407FEFDCF8EB574
:100D300061E08AE00E94BD0960E08AE00E94BD098E
:100D40000F5F1F4F0830110541F40894A11CB11C1E
:100D50008FE1A816B104E9F018C0C80123E0880F9C
:100D6000991F2A95E1F7EC01CC5FDE4FDC01AC570F
:100D7000BE4FFC01EC5BFE4F8FEFD82E7FEFE72ECE
:100D80006FEFF62E20E030E084CFCA2C00E010E0B8
:100D9000E4CFDF91CF911F910F91FF90EF90DF9003
:100DA000CF90BF90AF9008958BE292E00E949E0A90
:100DB00061E08DE00E944C0961E08AE00E944C09EC
:100DC00061E08BE00E944C0960E08CE00E944C09DD
:100DD00061E089E00E944C0960E08AE00E94BD0960
:100DE00060E08BE00E94BD0960E08DE00E94BD09DB
:100DF0000E9474036AE070E080E090E00E942209A3
:100E000040E060E080E00E94C3000E9496030895E5
:100E10000E94E8080E94D4060E94D605FDCFCF9319
:100E2000DF93992733E0880F991F3A95E1F7EC019A
:100E3000CC5FDE4FDC01AC5BBE4FFC01EC57FE4FDC
:100E400080E069934D9321938F5F8830D1F7DF91D4
:100E5000CF910895EF92FF920F931F93CF93DF935B
:100E6000EE24FF243FC049934D9341938F5F883018
:100E7000D1F72F5F3F4F2830310519F510E00E9460
:100E80003C061F5F1530D9F70894E11CF11C80E285
:100E9000E816F104E1F126C009930D9301938F5FE9
:100EA0008830D1F72F5F3F4F28303105F9F410E03B
:100EB0000E943C061F5F1530D9F701500F3F59F1D2
:100EC00027C0C90153E0880F991F5A95E1F7EC013B
:100ED000CC5FDE4FDC01AC5BBE4FFC01EC57FE4F3C
:100EE00080E0C1CF4E2D20E030E0EBCFC90143E0E0
:100EF000880F991F4A95E1F7EC01CC5FDE4FDC01CA
:100F0000AC5BBE4FFC01EC57FE4F80E0C5CF0FE15C
:100F100020E030E0EBCFDF91CF911F910F91FF9058
:100F2000EF900895CF93DF939927EC01CC5FDE4FCC
:100F3000DC01AC5BBE4FFC01EC57FE4F80E06883E8
:100F40004C9320838F5F2896189638968830B9F78F
:100F5000DF91CF9108951F920F920FB60F92112437
:100F6000AF92BF92CF92DF92EF92FF920F931F93B7
:100F70002F933F934F935F936F937F938F939F93A1
:100F8000AF93BF93CF93DF93EF93FF938FEC9EEFDD
:100F9000909385008093840060E089E00E94BD0901
:100FA000AA24BB247CC08881C81650F481E090E05C
:100FB000022E02C0880F991F0A94E2F78095D8226A
:100FC0008081C81650F481E090E0022E02C0880FA4
:100FD000991F0A94E2F78095E8228C91C81650F484
:100FE00081E090E0022E02C0880F991F0A94E2F778
:100FF0008095F8222F5F3F4F219611963196283029
:10100000310589F660E08AE00E94BD09FEBC0DB49E
:1010100007FEFDCF8EB5EEBC0DB407FEFDCF8EB53D
:10102000DEBC0DB407FEFDCF8EB581E090E0002E52
:1010300002C0880F991F0A94E2F78EBD0DB407FE17
:10104000FDCF8EB561E08AE00E94BD0960E08AE0D4
:101050000E94BD090F5F1F4F0830110541F408942D
:10106000A11CB11C8FE1A816B104C9F41CC0C801B1
:1010700023E0880F991F2A95E1F7EC01CC5FDE4F42
:10108000DC01AC57BE4FFC01EC5BFE4F8FEFD82E5E
:10109000EE24EA946FEFF62E20E030E084CFCA2CE5
:1010A00000E010E0E4CF61E089E00E94BD09FF911B
:1010B000EF91DF91CF91BF91AF919F918F917F91F0
:1010C0006F915F914F913F912F911F910F91FF90E1
:1010D000EF90DF90CF90BF90AF900F900FBE0F902A
:1010E0001F9018951F920F920FB60F9211242F93F5
:1010F0008F939F93AF93BF938091C6019091C70147
:10110000A091C801B091C9018050904CAF4FBF4F22
:101110008093C6019093C701A093C801B093C90101
:1011200027C08091C6019091C701A091C801B091DC
:10113000C90180589E43A040B0408093C60190935F
:10114000C701A093C801B093C9018091CA019091D1
:10115000CB01A091CC01B091CD010196A11DB11D93
:101160008093CA019093CB01A093CC01B093CD01A1
:101170008091C6019091C701A091C801B091C901A9
:1011800081589E43A040B04060F6BF91AF919F91BF
:101190008F912F910F900FBE0F901F9018952FB722
:1011A000F8946091CA017091CB018091CC0190912B
:1011B000CD012FBF0895019751F0880F991F880F17
:1011C000991F02972FB7F8940197F1F72FBF089551
:1011D000789484B5826084BD84B5816084BD85B512
:1011E000826085BD85B5816085BDEEE6F0E08081D9
:1011F00081608083E1E8F0E080818260808380818B
:1012000081608083E0E8F0E0808181608083E1EBB1
:10121000F0E0808184608083E0EBF0E08081816099
:101220008083EAE7F0E0808184608083808182604F
:101230008083808181608083808180688083109238
:10124000C1000895EF92FF920F931F937B018C01D1
:101250008FB7F8944091CA015091CB016091CC01B5
:101260007091CD018FBF2FB7F8948091CA019091F2
:10127000CB01A091CC01B091CD012FBF841B950B68
:10128000A60BB70B8E159F05A007B10760F31F9142
:101290000F91FF90EF900895282F3327C9018557AC
:1012A0009F4FFC01C895902D29583F4FF901C895D3
:1012B000802D882389F0E82FFF27E859FF4FC89534
:1012C000E02DFF27662329F4808190958923808370
:1012D00008958081892B80830895482F5527CA015E
:1012E00081569F4FFC01C895202DCA0185579F4FFD
:1012F000FC01C895902D49585F4FFA01C895302DD3
:10130000332319F480E090E00895222331F1233053
:1013100021F4809180008F7705C0243031F48091D2
:1013200080008F7D8093800018C0213019F484B52F
:101330008F7704C0223021F484B58F7D84BD0DC029
:10134000263021F48091B0008F7705C0273029F432
:101350008091B0008F7D8093B000E32FFF27EE587F
:10136000FF4FC895E02DFF27808120E030E08923E2
:1013700011F021E030E0C9010895482F5527CA0136
:1013800081569F4FFC01C895202DCA0185579F4F5C
:10139000FC01C895902D49585F4FFA01C895302D32
:1013A0003323C9F1222331F1233021F480918000CD
:1013B0008F7705C0243031F4809180008F7D809339
:1013C000800018C0213019F484B58F7704C0223012
:1013D00021F484B58F7D84BD0DC0263021F4809129
:1013E000B0008F7705C0273029F48091B0008F7D41
:1013F0008093B000E32FFF27E359FF4FC895E02DFE
:10140000FF27662329F4808190958923808308959E
:101410008081892B808308956F927F928F929F9213
:10142000AF92BF92CF92DF92EF92FF920F931F93F2
:10143000CF93DF93CDB7DEB739014A0129893A89C5
:101440004B895C8966197709880999092A193B092A
:101450004C095D090E94230DE618F70808091909CF
:10146000A80197010E94550D2A0D3B1D4C1D5D1DC5
:10147000CA01B901DF91CF911F910F91FF90EF90B9
:10148000DF90CF90BF90AF909F908F907F906F90A4
:101490000895AF92BF92CF92DF92EF92FF920F9397
:1014A0001F935B016C01611571058105910529F49C
:1014B00060E070E080E090E01AC00E94F80A7C01D1
:1014C0000E94F80A0027F7FC0095102F8701FF24DF
:1014D000EE24AA2797FDA095BA2FE80EF91E0A1F41
:1014E0001B1FC801B701A60195010E94550D1F9150
:1014F0000F91FF90EF90DF90CF90BF90AF90089545
:10150000EF92FF920F931F937B018C016217730779
:101510008407950764F4261B370B480B590BCA0147
:10152000B9010E94490AE60EF71E081F191FC801DB
:10153000B7011F910F91FF90EF900895009711F060
:101540000E94FD0A0895A0E0B0E0E9EAFAE00C94F8
:10155000AE0DEC01A880B980CA80DB80A114B10473
:10156000C104D10449F482E4E82E8EECF82E8CE01C
:10157000082F8FE1182F2EC0C601B5012DE133EFE2
:1015800041E050E00E94550D27EA31E440E050E090
:101590000E94230D7B018C01C601B5012DE133EFC3
:1015A00041E050E00E94550DCA01B90124E13BE041
:1015B00040E050E00E94230DE61AF70A080B190BD1
:1015C00017FF08C08FEF9FEFAFEFBFE7E80EF91EE0
:1015D0000A1F1B1FE882F9820A831B83C7019F77BA
:1015E000EAE0CDB7DEB70C94CA0D0E94A30A0895B5
:1015F00080E091E00E94A30A0895AA27BB27809368
:10160000000190930101A0930201B093030108959A
:101610005058BB27AA270ED079C16AD130F06FD1BC
:1016200020F031F49F3F11F41EF45FC10EF4E095F9
:10163000E7FB55C1E92F7BD180F3BA176207730727
:101640008407950718F071F49EF593C10EF4E095A8
:101650000B2EBA2FA02D0B01B90190010C01CA016C
:10166000A0011124FF27591B99F0593F50F4503E17
:1016700068F11A16F040A22F232F342F4427585F09
:10168000F3CF469537952795A795F0405395C9F721
:101690007EF41F16BA0B620B730B840BBAF09150D9
:1016A000A1F0FF0FBB1F661F771F881FC2F70EC078
:1016B000BA0F621F731F841F48F48795779567954B
:1016C000B795F7959E3F08F0B3CF9395880F08F034
:1016D0009927EE0F9795879508950CD017C10FD1D4
:1016E00040F006D130F021F45F3F19F0F8C05111FD
:1016F00041C1FBC01CD198F39923C9F35523B1F321
:10170000951B550BBB27AA2762177307840738F070
:101710009F5F5F4F220F331F441FAA1FA9F333D0CF
:101720000E2E3AF0E0E830D091505040E695001C83
:10173000CAF729D0FE2F27D0660F771F881FBB1F3F
:10174000261737074807AB07B0E809F0BB0B802D19
:10175000BF01FF2793585F4F2AF09E3F510568F065
:10176000BEC008C15F3FECF3983EDCF386957795E9
:101770006795B795F7959F5FC9F7880F911D969567
:10178000879597F90895E1E0660F771F881FBB1FC3
:10179000621773078407BA0720F0621B730B840B70
:1017A000BA0BEE1F88F7E095089504D06894B11144
:1017B000E1C00895C4D088F09F5790F0B92F9927C1
:1017C000B751A0F0D1F0660F771F881F991F1AF04C
:1017D000BA95C9F712C0B13081F0CBD0B1E008950D
:1017E000C8C0672F782F8827B85F39F0B93FCCF38E
:1017F000869577956795B395D9F73EF49095809542
:10180000709561957F4F8F4F9F4F0895E89409C061
:1018100097FB3EF490958095709561957F4F8F4F23
:101820009F4F9923A9F0F92F96E9BB279395F69539
:10183000879577956795B795F111F8CFFAF4BB0FB7
:1018400011F460FF1BC06F5F7F4F8F4F9F4F16C01B
:10185000882311F096E911C0772321F09EE8872FA5
:10186000762F05C0662371F096E8862F70E060E061
:101870002AF09A95660F771F881FDAF7880F9695DA
:10188000879597F9089507D008F481E0089503D06B
:1018900008F48FEF0895990F0008550FAA0BE0E8A0
:1018A000FEEF16161706E807F907C0F01216130622
:1018B000E407F50798F0621B730B840B950B39F462
:1018C0000A2661F0232B242B252B21F408950A26C8
:1018D00009F4A140A6958FEF811D811D089597F908
:1018E0009F6780E870E060E008959FEF80EC0895C6
:1018F00000240A94161617061806090608950024EF
:101900000A9412161306140605060895092E039468
:10191000000C11F4882352F0BB0F40F4BF2B11F4DC
:1019200060FF04C06F5F7F4F8F4F9F4F089557FD3B
:101930009058440F551F59F05F3F71F04795880F3D
:1019400097FB991F61F09F3F79F0879508951216D4
:1019500013061406551FF2CF4695F1DF08C0161680
:1019600017061806991FF1CF869571056105089431
:101970000895E894BB2766277727CB0197F9089548
:101980000BD0C4CFB5DF28F0BADF18F0952309F0EB
:10199000A6CFABCF1124EECFCADFA0F3959FD1F332
:1019A000950F50E0551F629FF001729FBB27F00D0D
:1019B000B11D639FAA27F00DB11DAA1F649F662762
:1019C000B00DA11D661F829F2227B00DA11D621FB1
:1019D000739FB00DA11D621F839FA00D611D221F6B
:1019E000749F3327A00D611D231F849F600D211D4F
:1019F000822F762F6A2F11249F5750408AF0E1F0F2
:101A000088234AF0EE0FFF1FBB1F661F771F881F3A
:101A100091505040A9F79E3F510570F060CFAACF7A
:101A20005F3FECF3983EDCF3869577956795B79525
:101A3000F795E7959F5FC1F7FE2B880F911D96954F
:101A4000879597F90895629FD001739FF001829F57
:101A5000E00DF11D649FE00DF11D929FF00D839F3D
:101A6000F00D749FF00D659FF00D9927729FB00DDA
:101A7000E11DF91F639FB00DE11DF91FBD01CF01ED
:101A80001124089597FB092E07260AD077FD04D06C
:101A900027D006D000201AF4709561957F4F0895E5
:101AA000F6F7909581959F4F089597FB092E05268F
:101AB0000ED057FD04D028D00AD0001C38F4509521
:101AC0004095309521953F4F4F4F5F4F0895F6F762
:101AD00090958095709561957F4F8F4F9F4F08959A
:101AE000AA1BBB1B51E107C0AA1FBB1FA617B70744
:101AF00010F0A61BB70B881F991F5A95A9F7809560
:101B00009095BC01CD010895A1E21A2EAA1BBB1B22
:101B1000FD010DC0AA1FBB1FEE1FFF1FA217B307B9
:101B2000E407F50720F0A21BB30BE40BF50B661FCF
:101B3000771F881F991F1A9469F760957095809593
:101B400090959B01AC01BD01CF0108952F923F926A
:101B50004F925F926F927F928F929F92AF92BF92BD
:101B6000CF92DF92EF92FF920F931F93CF93DF9369
:101B7000CDB7DEB7CA1BDB0B0FB6F894DEBF0FBEC6
:101B8000CDBF09942A88398848885F846E847D8413
:101B90008C849B84AA84B984C884DF80EE80FD8015
:101BA0000C811B81AA81B981CE0FD11D0FB6F8948B
:0C1BB000DEBF0FBECDBFED010895FFCFDA
:041BBC000100000024
:00000001FF
